:020000040800F2
:10200000C8040020854000085F3200086D320008D7
:1020100000000000000000000000000000000000C0
:102020000000000000000000000000007132000805
:102030000000000000000000733200086132000858
:10204000DF2F0008000000008B3D0008234000083F
:102050002F400008A9400008AB400008AD40000830
:1020600000000000AF40000805230008B140000850
:10207000B3400008B5400008B74000080000000069
:10208000B9400008BB40000800000000BD40000847
:10209000BF400008C1400008C3400008C540000818
:1020A000C7400008C9400008CB400008CD400008E8
:1020B000CF4000080121C006C00E8140B948016030
:1020C000704700B5BFF34F8FB748B8490860BFF3FA
:1020D0004F8F00BFFDE700B589B00020B4490870FC
:1020E000072000F000FE002000F0FDFD002301228B
:1020F0000B219020C00500F09EFE00230122082144
:102100009020C00500F097FE01220B219020C00511
:1021100000F034FF012208219020C00500F02EFFBE
:10212000012000900323022209219020C00500F025
:10213000BFFE01200090032302220A219020C00547
:1021400000F0B6FE9B499C4800F02AFF9A4800F038
:1021500041FF102001900020029080200390002079
:10216000049000200590002006900020079001A90F
:10217000924800F035FF002001900020029080205E
:1021800003900020049000200590002006908020FD
:102190008001079001A9B24800F022FF01210A2026
:1021A00000F04CFF0A20FFF785FF01210A2000F014
:1021B00045FF0A20FFF77EFFD04800780121014348
:1021C000CE480170CD480078DF210140CB48017036
:1021D000CA480078FB210140C8480170C748007810
:1021E000F7210140C548017009B000BD80B5C34862
:1021F00000780100C907C90F002951D000F0D8FFAD
:1022000000280BD0BD48007804210143BB48017071
:10221000BA48007808210143B8480170B7480078EF
:10222000C0B200090100C907C90F00292ED100F072
:10223000D5FF8C490860B1480078C0B28009010020
:10224000C907C90F002902D0002059490870584811
:102250000078012802D100F00FFA27E054480078F6
:10226000022802D100F086FA20E0514800780028C8
:1022700002D100F049F919E0A0480078202101437B
:102280009E48017000204A4908700FE000F0A6FF48
:1022900074490968401A152808D3FFF712FF05E0B2
:1022A00096480078202101439448017001BD00B593
:1022B00001000020C9B200290AD190490978C9B2A9
:1022C00049090A00D207D20F002A10D001200EE0DF
:1022D000C9B202290AD189490978C9B289090A0013
:1022E000D207D20F002A02D0012000E00020C0B2A5
:1022F00000BD824800780100C9B2C9080800C007C3
:10230000C00F704780B57D480078C0B20009010059
:10231000C907C90F002927D0794800682021084043
:1023200077490860002812D0764800684006FBD53F
:10233000224800680221884320490860C448006898
:1023400020210143C248016000F08EF828E01B48BC
:1023500000680821884319490860BD480068802149
:102360000143BB4801601BE0144800680821884312
:102370001249086011480068022188430F4908602B
:10238000B3480068802109010143B1480160B048A9
:102390000068802189000143AD48016000F064F8C5
:1023A00001BD000000E100E00400FA050CED00E0D2
:1023B0002C08002081060000003801401C0002406B
:1023C00010B504004D480078102101434B480170BE
:1023D00001220B219020C00500F0D0FD0122082130
:1023E0009020C00500F0CAFD002003E00021994ABA
:1023F0001154401CFF28F9D99748006801218843EF
:10240000954908601648006801218843144908600E
:102410009248046092489349086093489349086041
:102420008D480068022101438B4801608A4800689A
:1024300008210143884801608D480068402101431C
:102440008B48016084480068012101438248016093
:10245000C148006880210143BF48016010BD0000F1
:1024600030000240E407002080B524480078EF21C6
:10247000014022480170002208219020C00500F090
:102480007DFD00220B219020C00500F077FD00208B
:1024900003E000216F4A1154401CFF28F9D96E480F
:1024A0000068012188436C490860AC48006801213C
:1024B0008843AA49086080204000A9490860A948CB
:1024C000A94908606348A9490860A4480068022136
:1024D0000143A2480160A1480068082101439F48C8
:1024E00001609E480068012101439C4801609A48B0
:1024F0000068402101439848016001BDDC070020CD
:10250000000002401C38014080B55A480078C0B233
:1025100040080100C907C90F002963D12920944947
:1025200008700020924948708820914988704B209B
:102530008F49C87053208E49087145208C494871D5
:1025400056208B4988714F208949C87100208849DD
:102550000872002086494872002085498872002050
:102560008349C8720020824908730020804948735B
:1025700000207F49887300207D49C87300207C4972
:10258000087430207A494874312079498874FF20D2
:102590007749C874FF2076490875FF20744948754B
:1025A00089207349887576207149C875002004E038
:1025B000FF216F4A12181176401C1328F8D300F03F
:1025C0005DF9AD490860AC480068FFF7F9FE29489D
:1025D0000078022101432748017000F0FFFDCB493C
:1025E000086034E000F09AF9012829D1C848407801
:1025F000BB2802D1FFF765FD29E0C548807888280F
:1026000016D1C348807DC249CA7DFF21C943114309
:10261000CA43904209D100F058FE002802D00120A0
:10262000BC49087000F03FFA11E000F025FA0EE016
:10263000F32802D1FFF745FDFCE700F01DFA06E0A4
:10264000022802D100F018FA01E000F0F4F901BD0F
:1026500004000240C80500201C0002402000024087
:102660002838014024000240C8040020280002400D
:1026700020380140DC07002080B5A7480078C0B2B0
:1026800040080100C907C90F00293AD10A2038497A
:1026900008700020364948700620354988700020AF
:1026A0003349C8700020C04300F0DDFE010E304AFF
:1026B00011710100090C2E4A5171010A2C4A9171C5
:1026C0002B49C87100202A49087200202849487205
:1026D00000202749887200202549C87200F0CEF8F2
:1026E0006549086064480068FFF76AFE8A48007818
:1026F000022101438848017000F070FD83490860A1
:1027000029E000F00BF9012823D181484078BB284B
:1027100002D1FFF7D6FC1EE07D48807886280DD1D7
:102720007B4800F0D3F9002802D000F0BCF901E0AA
:1027300000F0A2F90220774908700CE0F92805D1D1
:1027400000207449087000F0AEF904E000F094F93C
:1027500001E000F070F901BD08380140300002408E
:102760003400024024380140380002403C0002405E
:102770004807002080B568480078C0B240080100D2
:10278000C907C90F002935D10720BA4908700020B0
:10279000B84948705220B74988703320B549C8708D
:1027A0003120B44908713020B24948713120B14913
:1027B000887100F0A3FD0100AE4AD171C143AD485C
:1027C000017255480078FB2101405348017000F028
:1027D00055F82949086028480068FFF7F1FD4E4880
:1027E0000078022101434C48017000F0F7FC474992
:1027F00008603FE000F092F8012839D14448407861
:10280000BB2802D1FFF75DFC34E041488078F02816
:102810001BD13F48C078522814D101203D4908708F
:102820003D480078C0B280080100C907C90F0029DF
:1028300005D139480078F72101403748017000F090
:1028400032F917E000F018F914E0F92805D100F08A
:102850002AF900202F4908700CE0862805D100F0E5
:1028600022F901202B49087004E000F005F901E08D
:1028700000F0E1F801BD0000E807002038B50124B0
:102880000220A849087000251CE07A48405DC0B2CB
:102890000009C0B200F008FEA24902226A4389186A
:1028A00048707448405D0007000F00F0FDFD9D4931
:1028B00002226A4389188870002D02D06D48405D5D
:1028C00024186D1C6B480078401CA842DDD2E04300
:1028D0000400E4B2200900F0E7FD924902226A43B5
:1028E000891848702007000F00F0DEFD8D49022294
:1028F0006A438918887003208A4902226A4389182A
:10290000C870022045432D1D280032BDE00700207D
:10291000C80600202C080020DC070020F8B50020A5
:10292000002700E07F1CFF2F07DC7F4AD25D032ACF
:10293000F8D1390000227C4BDA55FF2F65DC4F1EA1
:1029400000E07F1E002F61D4774AD25D022AF8D1C1
:102950000020754AD055CE1B761C083E3800401C1E
:10296000C0B20100491CC9B26F4A515C6E4A105C8A
:1029700000F04EF86D490870F00708D47008001F89
:10298000792804D2700869490978884201D0022068
:102990003CE0760801243800C01CC0B20100491C8C
:1029A000C9B2614A515C604A105C00F031F85F497D
:1029B00048705E4840782418002518E03800401D13
:1029C000022169434018C0B20100491CC9B2564AED
:1029D000515C554A105C00F01BF854494919887045
:1029E000B54203D251484019807824186D1CAE427C
:1029F000E4D2E0430400E4B24C4880198078844279
:102A000001D0022000E0012000E00020C0B2F2BDB1
:102A100038B502000D0000201000C0B200F02EFDFD
:102A2000000104002800C0B200F028FD01002000D1
:102A30004018C0B232BD80B500F0D0FB3C490968F7
:102A4000401A652814D33B480068401C3949086087
:102A500038480068052805D33748007840210143ED
:102A60003548017034480078FD210140324801703A
:102A700001BD00004807002000B530480068401C38
:102A80002E4908602D480068052805D32A4800789B
:102A9000402101432848017027480078FD2101406A
:102AA0002548017000BD002024490860002021490C
:102AB000086021480078FD2101401F4801701E4830
:102AC0000078BF2101401C480170704710B5040018
:102AD000E07E227FFF21C9431143CA4390421DD1AA
:102AE00015490978C9B2C9080A00D207D20F002ACD
:102AF00002D100F011FC03E000F000FC00F00CFC3F
:102B0000E07800062179090440186179090240182B
:102B1000A179401800F006FC012000E00020C0B2BE
:102B200010BD0000C8040020C8050020C806002011
:102B3000E0070020EC070020DC070020F007002061
:102B400080B500F00DF89949994A126812091207E8
:102B5000120F895CC840974908609648006802BD1A
:102B600010B50020002100240024002490480068B3
:102B70000C210140042902D0082902D017E08E4C14
:102B800016E08E49820C1207120F8C5C8C498D4A1C
:102B900012681207120F895CC00305D5864800F041
:102BA0000EFD6043040001E08748444300E0824C8E
:102BB000200010BD85480068012101438348016061
:102BC0007B48006882490140794801607F4800687D
:102BD000804901407D4801607C4800687E49014091
:102BE0007A480160724800687C4901407048016081
:102BF000744800680F21884372490860784800686B
:102C00001321884376490860764800680100C907A7
:102C1000C90F74480160002073490860704700B50F
:102C20006A48006871490140684801606748006867
:102C30008001FBD4634800680F2188436149086024
:102C4000604800685F490860594800686849014069
:102C50005748016056480068A02189030143544841
:102C600001605A48006880214904014357480160C7
:102C7000564800688001FBD55E4800680121014389
:102C80005C4801604A480068F02188434849086070
:102C900047480068464908604C4800688001FBD5F9
:102CA0004348006803218843414908604048006860
:102CB000022101433E4801603D4800680C2101406B
:102CC0000829F9D13A4800684B4901403848016069
:102CD00037480068364908604848006801210143C8
:102CE0004648016000BD00B5C0B2012807D1444884
:102CF00000688021890201434148016055E0C0B26B
:102D0000022807D13E4800688021C90201433C489F
:102D100001604AE0C0B2032807D139480068802129
:102D200009030143364801603FE0C0B2042807D1DF
:102D3000334800688021490301433148016034E091
:102D4000C0B2052807D12E4800688021C90301437D
:102D50002B48016029E0C0B2062807D12948006845
:102D60008021C9030143274801601EE0C0B2072843
:102D700007D1244800688021C9010143214801602E
:102D800013E0C0B2002806D11D48006801210143AC
:102D90001B48016009E0C0B2082806D11948006844
:102DA0008021090101431748016000BD444000082B
:102DB00004100240C400002000127A0054400008B1
:102DC000644000082C10024000093D000010024041
:102DD0000CB8FF00FFFFF6FEFFFFFBFFFFFFC0FF89
:102DE000301002403410024008100240FFFFFFFE86
:102DF000FFFFC2FF00200240FFF8FFFF0C1002405F
:102E0000141002401810024030B403680324022555
:102E10004D43AC40A3430360C368032402254D43E4
:102E2000AC40A343D2B2022461438A401A43130048
:102E3000C36030BC704770B50468032502264E435A
:102E4000B540AC432600012402254D43AC40344339
:102E500004608468032502264E43B540AC43DBB2D0
:102E600002254D43AB4023431C008460446801238A
:102E70008B409C43112A12D1220001248C40144320
:102E80004460C468032202234B439A4094432300C6
:102E90000124022251438C401C43C46007E044607B
:102EA000C4680322022359438A409443C46070BD1E
:102EB000F0B5059CC9B208290CDA066A0F2504276B
:102EC0004F43BD40AE4304254D43AC403443260040
:102ED000066211E0466A0F27BC460D00083D042734
:102EE0007D436746AF40BE430D00083D04277D4348
:102EF000AC403443260046620668032402254D4355
:102F0000AC40A6433500022602244C43A6402E4383
:102F100006608668032402254D43AC40A643DBB21D
:102F200002244C43A34033431E00866046680123BD
:102F30008B409E43122A12D1320001268E40164346
:102F40004660C668032202234B439A4096433300EF
:102F50000126022251438E401E43C6600DE04660AA
:102F6000C668032202234B439A409643330001264E
:102F7000022251438E401E43C660F0BD00B5D2B25E
:102F8000002A03D001228A40826103E0012210312D
:102F90008A40826100BD026901208840104070476C
:102FA000002202600268084B134303604268074B2B
:102FB00013404360C1604168054A0A40426081682D
:102FC0002A229143816070470C800000FFCFFFFFF1
:102FD000FFB7FFFF016801220A4302607047FEE766
:102FE00010B4026801239A43026003681A000A4B76
:102FF00013401A000B684C681C438B682343CC6851
:103000001C430B6923434C691C438B6923431343C3
:10301000036010BC704700BF0FC0FFFF80B5401EAB
:103020002749086000210020C04300F007F8002075
:103030002449086007202449086001BDF0B540B26A
:10304000002821D5214B40B20207120F083A9208FE
:10305000042462431D4C40B205072D0F083DAD0806
:10306000042675436459FF258607B60F08277E435B
:10307000B540AC438901C9B28007800F0825684379
:103080008140214399501AE0114A40B28308042438
:103090006343D258FF238407A40F08256C43A34041
:1030A0009A438901C9B283079B0F0824634399405F
:1030B0001143074A40B28008042358431150F0BD21
:1030C00014E000E018E000E010E000E01CED00E09B
:1030D00000E400E080B500203B4908703B480078E0
:1030E000FD2101403948017000F078F83849401856
:1030F00038490860354800780121014333480170A0
:1031000001BD10B530480478052000F02DFB0028E3
:1031100003D000202C4908702BE0012000F024FB94
:10312000002803D004202849087022E0002000F085
:103130001BFB002803D001202349087019E003205D
:1031400000F012FB002803D002201F49087010E095
:10315000042000F009FB002803D003201A4908705E
:1031600007E0022000F000FB002802D005201649ED
:10317000087015480078E4B2844203D000F02EF8BD
:103180001449086000F02AF812490968401A1249E7
:10319000884206D30D480078FD2101400B4801709C
:1031A00005E00A480078022101430848017010BD7B
:1031B000064800780100C9B249080800C007C00FDE
:1031C00070470148007870472D080020180800203B
:1031D00018FCFFFF1C080020E90300002A480068D3
:1031E000704780B5002009E08100284A89180968E5
:1031F0008022920504234343D150401C3028F3D34E
:1032000000F09CFBFFF70BFD00F034F8FFF798FC93
:10321000FA21890000F0D3F9FFF700FF0021002018
:10322000C043FFF70BFF0120FFF75DFD0220FFF712
:103230005AFD0520FFF757FD0323012206211448FC
:10324000FFF7F9FD01BD80B500F082FB01BD80B53F
:1032500000F093FB01BD80B5FFF7ACFC01BD7047EA
:1032600009480068401C08490860704700B5FEE73F
:103270007047704707480068032188430100032016
:103280000843044908607047200800200020000817
:10329000001400480000014000202549087000206B
:1032A00024490860002024490860704700B50100E7
:1032B0000020C9B2032905D11F490968002902D19C
:1032C000012000E00020C0B200BD00B5062805D0F6
:1032D000052803D0072801D0042803D11649086027
:1032E000012003E00020144908600020C0B200BDA6
:1032F0001148006870470E480078704780B5FFF7A6
:1033000057FF002802D00A48007801E0FFF759FF74
:10331000C0B200F02FF802BD80B500F00FF80449EC
:10332000087001BD03490860704702480068704793
:103330002E080020240800202808002000B581075E
:1033400001D5052014E0C10701D5042010E0810655
:1033500001D503200CE0010701D5022008E0C106D9
:1033600001D5022004E0400701D5012000E0002043
:10337000C0B200BD00B5C0B2032801D1202014E0C6
:10338000C0B2022801D108200FE0C0B2012801D14B
:1033900004200AE0C0B2042801D1012005E0C0B237
:1033A000052801D1022000E0002000BD00B5BFF3D8
:1033B0004F8F2F482F490860BFF34F8F00BFFDE7A5
:1033C00080B5002000F0FAF9002809D1002000F0B3
:1033D00032FB002804D10020FEF769FF002801D04D
:1033E000FFF7E4FF012000F0E9F9002809D10120EE
:1033F00000F021FB002804D10120FEF758FF00282F
:1034000006D01D480068012101431B48016005E00A
:103410001948006801218843174908600220FEF717
:1034200046FF002806D014480068022101431248D4
:10343000016005E010480068022188430E490860D9
:103440000320FFF733FF002806D00B480068102147
:1034500001430948016005E00748006810218843DE
:103460000549086001BD044909680840704700002B
:103470000400FA050CED00E0D807002000B50100BB
:1034800000200800C0B2010030390A2902D23038C9
:10349000C0B208E0C0B201004139062902D2373873
:1034A000C0B200E0002000BD0007000F0149085C29
:1034B000704700007440000800B5002801D12020AA
:1034C0007CE0C10701D5002078E0810701D501200B
:1034D00074E0410701D5022070E0010701D5032007
:1034E0006CE0C10601D5042068E0810601D5052005
:1034F00064E0410601D5062060E0010601D5072001
:103500005CE0C10501D5082058E0810501D50920FE
:1035100054E0410501D50A2050E0010501D50B20FA
:103520004CE0C10401D50C2048E0810401D50D20F8
:1035300044E0410401D50E2040E0010401D50F20F4
:103540003CE0C10301D5102038E0810301D51120F2
:1035500034E0410301D5122030E0010301D51320EE
:103560002CE0C10201D5142028E0810201D51520EC
:1035700024E0410201D5162020E0010201D51720E8
:103580001CE0C10101D5182018E0810101D51920E6
:1035900014E0410101D51A2010E0010101D51B20E2
:1035A0000CE0C10001D51C2008E0810001D51D20E0
:1035B00004E0400001D51E2000E01F2000BD0022D5
:1035C000030A8B420BD203098B4219D243088B4268
:1035D0002ED2411A00D20146524110467047FF22B6
:1035E00009023FD012068B4205D3121209028B4208
:1035F00001D31212090203098B4219D300E0090A10
:10360000C3098B4201D3CB01C01A524183098B42BB
:1036100001D38B01C01A524143098B4201D34B01A4
:10362000C01A524103098B4201D30B01C01A524107
:10363000C3088B4201D3CB00C01A524183088B428E
:1036400001D38B00C01A524143088B4201D34B0077
:10365000C01A5241884200D3401A5241CFD201468B
:103660001046704708B500F08FFB08BD80B50122F9
:103670000021AB48FFF7C8FB01220A21A848FFF749
:10368000C3FB01220B21A648FFF7BEFB01220D213F
:10369000A348FFF7B9FB01220E21A148FFF7B4FBB5
:1036A00001220F219E48FFF7AFFBFFF797FD0A3875
:1036B0009C49086000209C4908609C4800780121D2
:1036C00001439A48017099480078FB2101409748CE
:1036D000017096480078FD2101409448017001BDB9
:1036E00010B5924800780100C907C90F002934D0ED
:1036F0008F480468FFF772FD8A490968401A0A2852
:103700001ED38B480468FFF769FD8649086000F006
:1037100077F800F0D0F8864908608548006800F026
:10372000A9F8002806D181480078042101437F4888
:10373000017005E07D480078FB2101407B48017065
:103740007B48006860407B4908607A480068784997
:10375000096801407748016005E07448007802215B
:1037600001437248017010BD00B5C0B2052801D1F7
:10377000202019E0C0B2012801D1022014E0C0B21B
:10378000002801D101200FE0C0B2032801D1082098
:103790000AE0C0B2042801D1102005E0C0B202281E
:1037A00001D1042000E00020614909680840002898
:1037B00001D0012000E00020C0B200BD00B5010032
:1037C0000020C9B201290AD158490978C9B289082B
:1037D0000A00D207D20F002A10D001200EE0C9B291
:1037E00000290AD151490978C9B249080A00D2070B
:1037F000D20F002A02D0012000E00020C0B200BD9C
:1038000010B5002400214648FFF7C5FB002802D16F
:103810002000012404430A214148FFF7BCFB002893
:1038200002D12000022404430B213D48FFF7B3FBE3
:10383000002802D12000042404430D213848FFF75A
:10384000AAFB002802D12000082404430E2134489A
:10385000FFF7A1FB002802D12000102404430F2110
:103860002F48FFF798FB002802D1200020240443B2
:10387000200010BD00B50100012000290BD008294F
:1038800014D0102912D0202910D001290ED00229DD
:103890000CD004290AD024490968491C224A116025
:1038A000214909680A2904D3002002E000211E4AA8
:1038B0001160C0B200BD30B501000B00002206E06F
:1038C0001C001D4804235343C3582343521C032A9E
:1038D000F6D31948C068034018000B00002206E028
:1038E0001D00154B042454431B592B40521C032A22
:1038F000F6D303431800104AD06002220AE00E4BB0
:10390000042454431B191B1F1B680B4C04255543EF
:103910006351521E002AF2D1074A116030BD0000E7
:10392000000400480008002004080020F4070020DC
:10393000F8070020FC070020C807002003480068A3
:10394000102101430148016070470000002002403F
:1039500000B50C480C4908600C480B490860002071
:103960000B4908600B480C4908600C4800680028A7
:10397000FBD10B480449086000BD094802490860B2
:1039800070470000CCCC00000030004055550000CE
:1039900004300040FF0F0000083000400C300040B1
:1039A000AAAA000080B50023012200219020C005B2
:1039B000FFF741FA0023012201219020C005FFF703
:1039C0003AFA0023012202219020C005FFF733FAC2
:1039D0000023012203219020C005FFF72CFA0023C9
:1039E000012204219020C005FFF725FA00220021C2
:1039F0009020C005FFF7C2FA002201219020C005E7
:103A0000FFF7BCFA002202219020C005FFF7B6FAAA
:103A1000002203219020C005FFF7B0FA0022042104
:103A20009020C005FFF7AAFAAE48007801210143B3
:103A3000AC48017001BD00B501000020C9B20029E9
:103A40000AD1A8490978C9B2C9080A00D207D20F19
:103A5000002A02D0012000E00020C0B200BD80B5E5
:103A60000120FFF700FD002803D01F2000F0BAF866
:103A7000B7E00220FFF7F7FC002804D11020FFF781
:103A8000F2FC00281CD0FFF7A9FBB7490968401ACF
:103A9000C82800D2A5E0FFF7A1FBB3490860914810
:103AA0000078C0B240080100C907C90F002903D03F
:103AB000002000F097F894E01F2000F093F890E0C9
:103AC000FFF733FC002865D0FEF713FC002861D116
:103AD000FFF76EFB00285DD182480078C0B28008F5
:103AE0000100C907C90F002928D0FFF777FB9E49BD
:103AF0000968401AC82826D37A480078C0B240081E
:103B00000100C907C90F002909D0002000F06AF898
:103B100074480078FD2101407248017009E0934823
:103B2000006800F05FF86F480078022101436D489B
:103B30000170FFF753FB8C49086004E0FFF7DBFBE3
:103B4000C0B200F09DF8FFF749FB89490968401AA7
:103B50008849884245D363480078C0B28008010094
:103B6000C907C90F002906D05E480078FB21014033
:103B70005C48017009E05B48007804210143594822
:103B8000017000F0B1F879490860FFF727FB784928
:103B9000086026E0FEF7ADFB002803D1FFF708FB25
:103BA00000280FD0FFF70DFBC0B200F069F84D48B8
:103BB0000078042101434B480170FFF70FFB6C496B
:103BC00008600EE0FFF797FBC0B200F059F84548D7
:103BD00000780421014343480170FFF7FFFA64496C
:103BE000086001BD10B50400E00606D400220021E3
:103BF0009020C005FFF7C2F905E0012200219020C6
:103C0000C005FFF7BBF9600706D40022022190200F
:103C1000C005FFF7B3F905E0012202219020C0059D
:103C2000FFF7ACF9200706D4002201219020C0053F
:103C3000FFF7A4F905E0012201219020C005FFF75C
:103C40009DF9E00706D4002204219020C005FFF76B
:103C500095F905E0012204219020C005FFF78EF9B7
:103C6000A00706D4002203219020C005FFF786F9A3
:103C700005E0012203219020C005FFF77FF910BD68
:103C800080B5C0B2002803D10420FFF7ABFF28E0C5
:103C9000C0B2022803D10120FFF7A4FF21E0C0B287
:103CA000012803D10820FFF79DFF1AE0C0B20428C5
:103CB00003D11020FFF796FF13E0C0B2032803D111
:103CC0000220FFF78FFF0CE0C0B2052803D10020CF
:103CD000FFF788FF05E00348007810210143014801
:103CE000017001BD0808002010B5FFF71EFB00247D
:103CF00000E0641C202C17D21F490968802252055D
:103D0000914209D01C490968002905D01A4909685F
:103D10004900194A116002E00121174A1160164951
:103D2000096801400029E4D013480068FFF7C4FB8C
:103D30000400202C16D2FFF7DBFA062804D10F4826
:103D400004214C4300590EE0FFF7D2FA052804D1B4
:103D50000B4804214C43005905E00A4804214C4318
:103D6000005900E0002010BD100800200C080020C1
:103D700014080020B80B0000C00000200C3E000812
:103D80008C3E00088C3D00087047FEE701000000F3
:103D900001000000040000000D0000000100000010
:103DA0000F000000070000000800000002000000F3
:103DB0000A0000000B0000000B00000011000000D2
:103DC000010000000E000000100000000D000000C7
:103DD00012000000130000000B0000000D000000A6
:103DE00016000000180000001A0000000D0000007E
:103DF0001B0000000D0000001D0000000D00000071
:103E000018000000020000001F0000000D0000006C
:103E10000D000000040000000D0000000100000083
:103E20000F000000070000000D000000020000006D
:103E30000A0000000B0000000B0000000B00000057
:103E40000B0000000E000000100000000300000046
:103E500012000000130000000B000000050000002D
:103E600016000000180000001A0000000800000002
:103E70001B0000000D0000001D0000001E000000DF
:103E800018000000020000001F00000001000000F8
:103E900001000000040000000D000000010000000F
:103EA000070000000A0000000B0000000B000000EB
:103EB0000E000000100000001200000013000000BF
:103EC0000B000000160000001800000018000000A1
:103ED0001A0000001B0000000600000006000000A1
:103EE0000600000006000000060000000F000000B1
:103EF0001D0000001D000000110000000200000075
:103F00000D0000000D0000000D00000070B4012144
:103F1000002213E00468001D0C4202D04D466D1EC5
:103F200064192260241D1B1F042BFAD225009E0752
:103F300001D52280AD1C0B4000D02A700368001D03
:103F4000002BE7D170BC704780B5FFF74AF9FFF747
:103F5000A3F9FEF7C0F8FFF789FBFFF723FDFFF792
:103F6000B9F8FFF770F9FFF772F9FFF7B9FBFFF740
:103F7000C8F8FEF73BF9FFF772FDFFF721FAF2E709
:103F800030B401210268001D002A0FD00368C31855
:103F9000446808300C4202D04D466D1E64191D68FD
:103FA00025601B1D241D121FECD0F8E730BC7047A4
:103FB00010B5074979441831064C7C44163404E0A6
:103FC000081D0A68891888470100A142F8D110BD70
:103FD000080000002800000035FFFFFF6803000014
:103FE000C80400200000000099FFFFFF0800000047
:103FF000B0000000C00000200000000000F00BF83E
:10400000002801D0FFF7D4FF002000BF00BFFFF75A
:104010009BFF00F002F80120704780B500F002F825
:1040200001BDFEE70746384600F002F8FBE7FEE771
:1040300080B500BF00BF024A11001820ABBEFBE7ED
:104040002600020000000000010203040102030434
:104050000607080902030405060708090A0B0C0DE8
:104060000E0F10100102030405060708090A0B0CC5
:104070000D0E0F1030313233343536373839414276
:1040800043444546014880470148004757320008ED
:104090009540000800BF00BF00BF00BFFFF7AEFFA4
:1040A0000100000000127A00FEE7FEE7FEE7FEE7EF
:1040B000FEE7FEE7FEE7FEE7FEE7FEE7FEE7FEE7D8
:1040C000FEE7FEE7FEE7FEE7FEE7FEE7FEE7FEE7C8
:04000005080040951A
:00000001FF
